:10000000830100308A005528FC0003088301E800C2
:100010000408E90083018C1E2E2883168C1E2E28CE
:1000200083121A08E70098181728181D19281812A3
:10003000181667080D3A031D232883168C128312A5
:10004000A301A30A4C282530220203182E282208D7
:100050002A3E8400831367088000A20A8B180B1EB7
:100060004C288312200B3C28A801A901051A3A2824
:10007000A1034B28A10A4B28851D051A4428A0017D
:10008000A00AA801A9014B28A508031D4A28A5011B
:10009000A50A4B28A5018B1003138312690884005D
:1000A00068088300FC0E7C0E090020308400683054
:1000B0005E208301862B04068001840A0406031D4A
:0400C0005B28003485
:0803F8006322632A8301E30084
:100400000510082B8301A4010130FE210D2A913033
:100410008301E500FD30E6006E2ACD308301D70070
:10042000F330D800DC2A85308301E500FF30E60098
:100430006E2A98308301D700E730D800DC2A2E30AE
:100440008301D700CF30D800DC2AF0308301D700F9
:100450008530D800DC2AE2308301E500FF30E60079
:100460006E2AFB308301E500FF30E6006E2AC330C0
:100470008301E500FF30E6006E2A2E308301E5009F
:10048000CF30E6006E2ADE308301D7000B30D80073
:10049000DC2ACF224D30592207220D30592200305C
:1004A0004F2C8312D90083169B001C141A08831248
:1004B00008008301D000831203130C1E5B2A50082E
:1004C00099000C120800DE308301D7000B30D800F1
:1004D000DC22DE30D7000B30D800DC2A830165082F
:1004E0008E0066088F0010140C1C742A10100C105B
:1004F00008008301D8008522F000F00EF030F005EE
:10050000700857088522700708008301D900413020
:10051000590203188D2AD0308E2AC930D9075908BC
:10052000080083018519080027082606031908001A
:10053000851712151F22121108008301051A0800E1
:10054000A008031D0800051EA32A2608A70085137E
:1005500008008301D0000A3050020318B12A30305D
:10056000B22A3730D0075008080003304F24003833
:10057000031D0800CF225630592207220D30592280
:1005800003304F2C8301D800C92AD80A58035122BE
:10059000F82283120313D703570FC52A08008301DB
:1005A0001A08D0001A08D0001A08D000A201A3012E
:1005B00083168C1683120800830157088E00580892
:1005C0008F001014E42A9D220C1CE32A10100C103A
:1005D000080002220630D7006730C2223A30F822E3
:1005E000210E0F39A922F82221080F39A922F82A51
:1005F0008301E2000A302402031CA40A2408093AF9
:10060000031D052BC030FE21132205146208082BA0
:100610008301E4000F3086056408F039860405156F
:1006200005110F308605640EF03986040515051195
:10063000372A8301E100222BE10A6103840083133E
:100640000008F822831203136108840083138008D2
:10065000031908001C2B8301851005100D220F3093
:10066000860530308604051505110722051505118C
:100670000722051505110F3086058616051505118B
:1006800007222830FE210C30FE210630FE2180306A
:10069000FE298301DA00F0009D265708F300580870
:1006A000F4005908F5007B27F3018030F400433053
:1006B000F50043277008DB007108DC007208DD00DC
:1006C0005B08F0005C08F1005D08F200080083019F
:1006D000250B0800CF224C305922072230305922F6
:1006E00007223630592207220D30592201304F247B
:1006F000CF224C3059220722303059220722413074
:10070000592207220D30592202304F2CBE232B23B1
:1007100002221030D7000030C2226322B522200B03
:10072000AD2BE9223D22A80A0319A90A2808323A6A
:100730002904031D8F2BCF22463059220722210E78
:100740000F39A9225922072221080F39A92259223B
:1007500007220D305922A0018F2B0222851DB52BB7
:1007600005170A30D7001030B92B05130630D70013
:100770001430C2226322492267238F2B0730830162
:100780009F00183083168500033086008113831282
:10079000A201A301203083169800903083129800A4
:1007A00033308316990083129A019A019A0110102E
:1007B000901610169010121192101214971517150A
:1007C000FF3083169200803083129500971617121F
:1007D000831601170B168C160B178B178312051730
:1007E0008513A801A901A001A501A701A601080080
:1007F00083015708F0005808F1005908F200BC279F
:100800007008DA00F0009D267008F3007108F4000B
:100810007208F500573084008313EF268312031308
:100820005A08303EDB002E30DC005708F300580831
:10083000F4005908F500F0012030F1004130F200D9
:100840007B27BC277008DA00F0009D26F3012030DA
:10085000F4004130F50043277008F3007108F400FC
:100860007208F500573084008313EF2683120313B8
:100870005A08303EDD005708F3005808F4005908C4
:10088000F500F001C830F1004230F2007B27BC27B0
:100890007008DA00303EDE00DF015B30192B830187
:1008A000D0000A30D200D301562C25225208031959
:1008B000D303D203520A0319530A0319622CA30863
:1008C0000319552C230B832E472EA6012B08D70086
:1008D0002A087922D1004E305102031C732C9A3021
:1008E0005102031C742C26142F08D7002D087922DE
:1008F000D10031305102031C812CAA305102031C5B
:10090000822CA6143408D70033087922D10066302F
:100910005102031C8F2CB4305102031C902C26155D
:100920003A08D70039087922D1001A305102031C45
:100930009D2CE7305102031C9E2CA6153D08D700C4
:100940003C087922D1001A305102031CAB2CE7304D
:100950005102031CAC2C26164008D7003F08792210
:10096000D10066305102031CB92CE7305102031C40
:10097000BA2CA6160222A508031DE02C2A08F8228C
:100980002B08F8222D08F8222E08F8223008F82229
:100990003108F8223308F8223408F8223608F82201
:1009A0003708F8223908F8223A08F8223C08F822D9
:1009B0003D08F8223F08F8224008F8229122812EB3
:1009C0000930D7002430C2223A30F8222B08D70051
:1009D0002A087922D100D701A030D8004030D900B0
:1009E000510849237008F3007108F4007208F500FB
:1009F000F001A030F1004030F20012277008D4005E
:100A00007108D5007208D6005408D7005508D800E0
:100A10005608D900F8235630F822261C122D213012
:100A2000F822912291226322A5080319013402229F
:100A30000930D7002D30C2223A30F8222E08D700D4
:100A40002D087922D100D701A030D8004030D9003C
:100A5000510849237008D4007108D5007208D600E7
:100A60005408D7005508D8005608D900F823563046
:100A7000F822A61C3E2D2130F82291226322A508DF
:100A80000319013402220930D7003630C2223A302D
:100A9000F8223408D70033087922D100D701A030DA
:100AA000D8004030D900510849237008D40071089B
:100AB000D5007208D6005408D7005508D80056084B
:100AC000D900F8235630F822261D692D2130F8224E
:100AD00091226322A5080319013402220930D700AC
:100AE0003F30C2223A30F8223708D7003608792240
:100AF000D100D701A030D8004030D9005108492397
:100B00007008D4007108D5007208D6005408D700C8
:100B10005508D8005608D900F8235630F822632229
:100B2000A5080319013402220930D7004830C22237
:100B30003A30F8223A08D70039087922D100D70193
:100B4000D8013F30D900510849237008F3007108DB
:100B5000F4007208F500F001F1013F30F2001227B5
:100B60007008D4007108D5007208D6005408D70068
:100B70005508D8005608D900F8234130F822A61DA0
:100B8000C42D2130F82291226322A50803190134D3
:100B900002220930D7005130C2223A30F8223D08F3
:100BA000D7003C087922D100D701D8013F30D900C5
:100BB000510849237008F3007108F4007208F50029
:100BC000F001F1013F30F20012277008D4007108E3
:100BD000D5007208D6005408D7005508D80056082A
:100BE000D900F8234130F822261EF92D2130F822B1
:100BF00091226322A5080319013402220930D7008B
:100C00005A30C2223A30F8224008D7003F087922F1
:100C1000D100D701A030D8004030D9005108492375
:100C20007008D4007108D5007208D6005408D700A7
:100C30005508D8005608D900F8235630F822A61EC9
:100C4000242E2130F82291226322A50801340222A9
:100C50000330D7006330C2222030F8224330F8221C
:100C60003A30F8222A08F8222B08F82201342030E2
:100C7000F8224630F8223A30F8222A08F8222B08C7
:100C8000F8222B08D7002A087922A100812E5008CB
:100C90000319652C013A0319272E033A0319372E3D
:100CA000013A0222D201D30152082A3E8400831362
:100CB0000008F822D20A0319D30A5308803AF00038
:100CC000803070020E3003195202031C542E63222E
:100CD000632202220F30D200D30152082A3E840040
:100CE00083130008F822D20A0319D30A5308803A62
:100CF000F000803070021B3003195202031C6D2E6D
:100D00006322632201340A30D7001A30C222003431
:100D1000840803190034720880008403710880007D
:100D20008403700880000034F101F201F301F01F28
:100D3000E42FF103F203F303DF2FF101F201F301DA
:100D4000E42FF801710D720DF60076080319AC2E30
:100D5000F80DF201F1170800F001F101F201003481
:100D6000F810740D750DF70077080319BC2E0318E1
:100D7000F814F501F4170800F701F301F401F50187
:100D8000080076080319AC2EF113F80C760CF2006B
:100D90000318F117882EF608031DDF2EF001F1016C
:100DA000F201882E72030319F00A0319F10A0319DC
:100DB000F20A0310F20CF10CF00CF60ACB2EF2083A
:100DC000031DD22E700871040319CE2EF11BC12E03
:100DD000F6030319CE2E0310F00DF10DE62E803030
:100DE000F5060008F000840A0008F100840A0008F3
:100DF000F200152F76087702031C092F031908004B
:100E00000310F20CF10CF00CF60A76087702FE2EB5
:100E10000310F50CF40CF30CF70A760877060319A7
:100E20000800082F8030F5068401A126B026FA2696
:100E3000781C222FF009F109F209F00A0319F10ACE
:100E40000319F20AF81C2C2FF309F409F509F30A27
:100E50000319F40A0319F50A7308F0077408031854
:100E6000740FF10775080318750FF207F801F21FE8
:100E7000CB2EF009F109F209F00A0319F10A03195E
:100E8000F20A7814CB2E8401A126B026F901FA01CA
:100E9000FB01F60803190800770803190800760219
:100EA000773EF600780CF8061830F5000310F90DBF
:100EB000FA0DFB0D7208031D652F74087102031DE6
:100EC000632F73087002031C6F2F7308F0027408FD
:100ED000031C740FF102031CF20379140310F00DCC
:100EE000F10DF20DF50B562F7908F0007A08F1009C
:100EF0007B08F200CB2E8401A126B026F901FA016D
:100F0000FB010730F5000310F40CF30C031C932FC6
:100F10007008F90771080318710FFA0772080318AF
:100F2000720FFB070310F00DF10DF20DF50B832F7F
:100F30000930F5009F2F0310FB0CFA0CF90C03107D
:100F4000F40CF30C031CAE2F7008F907710803189A
:100F5000710FFA0772080318720FFB07F50B9B2F2E
:100F60007A307707F607780CF8067908F0007A08E7
:100F7000F1007B08F200CB2E8401A126F301823020
:100F8000F607F61BAC2EF030F607F61BD82F1830FC
:100F900076020318AC2EF608031DD12F7818F2271D
:100FA0000800F6030310F00DF10DF20DF30DCB2F39
:100FB0000310F20CF10CF00CF60FD82FCE2FF31F0C
:100FC000E42F7814F227E52FF8018E30F600840123
:100FD000F3080319CB2E0310F30CF20CF10CF00CF8
:100FE000F60AE82F0310FF30F007F009031CF107A1
:100FF000F109031CF207F209031CF307F3090800C7
:02400E00703F01
:1042000054004D005800200031002E0030002000E6
:1042100042002E00560045004C004C004500200096
:104220004E004F00540020004C004F0043004B0054
:104230004500440043004F004D002E002000450083
:10424000520052004F005200430065006C006C00A9
:104250002000560061006C002E00520075006200C4
:10426000690020005000650061006B0056004300AB
:1042700058004F00200043006F006E00740046009D
:104280007200650071002000410064006A002E0089
:104290004C0061006D007000200048006500610066
:1042A0007400430065006C006C002000480065004D
:1042B00061007400390030004D0048007A00200091
:1042C000500057005200410044004A0020004300C3
:1042D0004F004E004600490047002000200020000B
:1042E00020002000200020002000200020002000CE
:00000001FF
